:1000000003308A002F2B0000CD306737653AEF367A
:10001000653A721D20100D050000A831A936EC309C
:100020006210CA2043244F103218B1193A10A006AA
:100030000A00D63C73366532EB3C203D20356532F4
:10004000EE377436693BF9316810EF39BA060A00A9
:10005000D63C73366532EB3C203D20356532EE37B9
:100060007436693BF9316810EF39BA060A00A013FB
:10007000200883168700831287130830F800402871
:100080000000F8175128F813B00C03188717031C49
:100090008713781751287813F80B44284F2800004D
:1000A00087173F308400840B53280000F81B432837
:1000B000781B4B280800831603178C170C140000BC
:1000C000000083120C087F3903199F280313A7002F
:1000D00003170D080313A80003170F080313A90043
:1000E0002708B0003720280803178D0003132908BC
:1000F00003178F0083168C170C1400000000831266
:100100000C0D0E0D7F3903199F280313A700031749
:100110000D080313A80003170F080313A9002708ED
:10012000B0003720280803178D0003132908031790
:100130008F008D0A03198F0A03135B28031703131B
:1001400008000830F80000008711A011200883166D
:10015000870000008312AC0D0712031CB52820167F
:10016000200883168700B9288312201220088316DE
:10017000870000008312A0152008831687008312D1
:10018000871DC028F80BA32800008711A0112008A4
:10019000831687000000831220162008831687002C
:1001A000000000008312A015200883168700831228
:1001B000871DD828F8010000071A78148711A011AC
:1001C0002008831687008312071220122008831646
:1001D0008700831208002830840083130008031965
:1001E000FE280230F800F701F70BF428F80BF3288B
:1001F0009730F700F70BFA28800BF128080020163B
:1002000020088316870000008312A015200883169B
:10021000870000008312071220122008831687002F
:10022000000083128711A0112008831687003C303C
:100230008312AC00A120AC01A1207030AC00A12041
:10024000201220088316870000008312A0152008C2
:10025000831687008312871D2B2900002F29000099
:100260002016200883168700000006308312A8009D
:10027000EB20201620088316870000008312A015AB
:10028000200883168700000083120712201220081E
:1002900083168700000083128711A011200883169F
:1002A00087003C308312AC00A1200130AC00A120BB
:1002B000E030AC00A1202012200883168700000047
:1002C0008312A0152008831687008312871D6629D4
:1002D00000006A290000201620088316870000000D
:1002E00006308312A800EB20201620088316870012
:1002F00000008312A01520088316870000008312D7
:10030000071220122008831687000000831287112D
:10031000A0112008831687003C308312AC00A12076
:100320000230AC00A120AC01A120201220088316CD
:10033000870000008312A01520088316870083120F
:10034000871DA0290000A42900002016200883167C
:100350008700000006308312A800EB208A110A12E1
:10036000AA2B201620088316870000008312A015F0
:10037000200883168700000083120712201220082D
:1003800083168700000083128711A01120088316AE
:1003900087003C308312AC00A1202B08AC00A120C8
:1003A000201220088316870000008312A015200861
:1003B000831687008312871DDB290000DF290000D8
:1003C00020162008831687000000831220162008BC
:1003D0008316870000008312A0152008831687006B
:1003E00000008312071220122008831687000000E5
:1003F00083128711A0112008831687003D308312D5
:10040000AC00A120F7010830AD007708AE0020163F
:1004100020088316870000008312A0152008831689
:1004200087008312871D122A071A0314071E031060
:10043000F80D0000A0112008831687008312871191
:10044000AD0B072A201620088316870000008312B0
:1004500007122E080319312A20122008831687005C
:1004600083120000A0152008831687008312871DC1
:10047000372A00008711A01120088316870000008A
:10048000831207122012200883168700780883122F
:10049000AB002B08F8000800B0012B08AF00B0003B
:1004A000AF012C082F07F8003008FA000318FA0AE9
:1004B0007808AD007A08AE002D08F8002E08F90083
:1004C00008000330AB00B1217808A7000430AB006E
:1004D000B1217808A8002708AB002808AC004C22FE
:1004E0007908AA007808A9002908F8002A08F90064
:1004F0008A110A12B22B0730AB00B1217808A7008D
:100500000830AB00B1217808A8002708AB00280804
:10051000AC004C227908AA007808A9002908F80044
:100520002A08F9008A110A12B72B0530AB00B12155
:100530007808A7000630AB00B1217808A80027088A
:10054000AB002808AC004C227908AA007808A90062
:100550002908F8002A08F9008A110A12BC2BAF01F9
:100560000408AE002F10831B2F14A81FBF2AAE173C
:100570002E1EAE0AA709A809A70A0319A80A280E61
:10058000F038AA00AA07E23EAB00323EAD002808D0
:100590000F39AB07AB07AD07E93EAC00AC07AC07C2
:1005A000270E0F39AC07AD07AC0DAD0DAD09AD0D84
:1005B00027080F39AD07AA0D0730A9000A30AD078B
:1005C000AC03031CDF2AAC07AB03031CE32AAB0715
:1005D000AA03031CE72AAA07A903031CEB2A293054
:1005E0008400831307302E052E1384032E05031D6C
:1005F000002B2E1A840A2E1A002B2030F7001D2BF8
:1006000084072D30040203192E170008F700031D7C
:10061000112B2E1B112B2E1A2B2BAE19112B203028
:100620001C2BAE1F192B2D30F70084032E13AE1395
:100630001D2BAE152E123030F707A8010408A700B5
:100640002810831B28147708B0003720270884005F
:10065000831328188317840A2E1F012B0800840196
:1006600083131F308305713083168F000F088312A8
:10067000A013200883168700831287178316031799
:100680000908C039890003131F129F120030031795
:1006900088008312870188018901FF300313A000BD
:1006A000831603170908C039890003131F129F120C
:1006B000003003178800831203131F139F13831640
:1006C0009F1383121F149412A01220088316870010
:1006D000831220162008831687008312A011200899
:1006E0008316870001308312940000308316940033
:1006F0000108C73908388100831290010030F800E2
:100700009200003083169200831220152008831671
:1007100087008312970183169B019C0101309D0085
:100720008312031787018801890104308D0000308E
:100730008F0003135B200D3003178D0000308F00F6
:1007400003135B20193003178D0000308F00031353
:100750005B20FF28283003178D0000308F00031323
:100760005B20612A7908A2007808A1007B2A790819
:10077000A4007808A300952A7908A6007808A500A7
:100780005830B00037203A30B00037202030B00069
:100790003720103084002208A8002108A700AF22CB
:1007A0002030B00037200D30B00037200A30B000C4
:1007B00037205930B00037202030B00037201030BB
:1007C00084002408A8002308A700AF222030B0002E
:1007D00037200D30B00037200A30B00037205A30B3
:1007E000B00037203A30B00037202030B00037203A
:1007F000103084002608A8002508A700AF2220306A
:10080000B00037200D30B00037200A30B00037205C
:100810000830A700FA30A800EB20A70B0A2CAA2B5F
:02082000630073
:04400E00F52CFF3F4F
:00000001FF
